:1020000000800020B12400009924000099240000E1
:1020100000000000000000000000000000000000C0
:1020200000000000000000000000000099240000F3
:1020300000000000000000009924000005250000B9
:10204000992400009924000099240000992400009C
:102050009924000099240000992400009D24000088
:10206000992400009924000099240000992400007C
:1020700099240000992400000924000099240000FC
:10208000992400009924000099240000592200009E
:102090000000000099240000992400009924000009
:1020A000992400009924000099240000992400003C
:1020B0000000000010B5064C2378002B07D1054B1B
:1020C000002B02D0044800E000BF0123237010BDA4
:1020D000A000002000000000FC4E0000044B10B5E2
:1020E000002B03D00349044800E000BF10BDC046E8
:1020F00000000000A4000020FC4E000010B50921E3
:10210000014800F079F910BDBC000020044B10B567
:102110001868C0B200F0C6FB024B186010BDC04684
:1021200000000020C000002010B5024800F09EF81A
:1021300010BDC046BC000020F7B50C27404E0193EF
:10214000335C04005BB20D0000924743002B2EDA93
:1021500000230B82EB7BDB09FCD1335D394A013371
:102160005BB23355335D12785BB2DB19934203DA0D
:10217000335D5BB20B2B34DD2F8ABFB2EB7BDB0907
:10218000FCD1314B3149186802F0DEFA304B04378C
:102190005843009B00090C3387424DD280B25B004C
:1021A0005853EB7BDB09FCD1FF33335540E0335C04
:1021B000244A5BB21278DB199342CEDA335C254AAB
:1021C0005BB2DB19DB009B5C5B06C6D5335C002190
:1021D0005BB2DB19DB00985C8006800E00F01CFC13
:1021E000BBE7335D1B4A5BB2DB19DB009B5C5B0624
:1021F00009D5335D01215BB2DB19DB00985C8006F9
:10220000800E00F009FC2A8A92B2EB7BDB09FCD13C
:10221000335D5BB2DF190F4BFF00DF197B68D3180A
:10222000009A9BB20C3252005353EB7BDB09FCD17A
:102230006B461B79AB73F7BDBFB25B005F53B0E772
:10224000C5000020C40000200400002040420F0010
:10225000204E0000C8000020002210B510230249C3
:102260001000FFF769FF10BD0030004270B50C4B45
:1022700005001C780B2C10D8621C1A70094B0470D6
:102280001868094902F060FA084BE4005843084B0B
:1022900000091C196060280070BDFF230370FAE775
:1022A000C40000200400002040420F00DC050000B4
:1022B000C8000020F7B50193037804000E00170052
:1022C0000B2B00D986E0C8B2012100F059FB3F2159
:1022D00032002078404DC3005E5D0A408E431643B5
:1022E0005E558823032296219B00DB1BDF171740D6
:1022F000FF18019B0901C91ACB1713405B189B10EB
:10230000BF10A37067700C2102F01EFA0C23C0B23C
:1023100043431A000C32D900695C490654D4013396
:102320009342F8D100284FD12C4B2D4A5A805A782D
:10233000D209FCD12B4E0232338893433380F37B96
:10234000DB09FCD101333380F37BDB09FCD133881B
:10235000DB07FCD433889BB233804023328813439D
:10236000338080233288DB001343338001233279AA
:1023700013433371F37BDB09FCD11B4B1B491868FA
:1023800002F0E2F90300FA2080005843000980B20D
:102390003083F37BDB09FCD18021154B0903D9671E
:1023A000C023C420134A5B00D150800013581B0285
:1023B0001B0A135010231160737332880E3B1343B2
:1023C0003380F37BDB09FCD140222378DB00E95C1E
:1023D0000A43EA542078FEBDC8000020000C0040EB
:1023E0001C400000003000420400002040420F006A
:1023F00004E100E000E100E09623882210B51B0113
:102400009200FFF757FF10BD10B5024800F075FEAF
:1024100010BDC0462801002013B51249124800F033
:10242000D5FB1249124800F0D1FB1249124800F0C6
:10243000CDFB1249124800F0C9FB1249124800F0C6
:10244000C5FB124C1249200000F0C0FB0123019390
:10245000023300930D220B3321000E4800F0C6FD1D
:1024600013BDC046000800426C030020000C00426F
:1024700074030020001000427C030020001400427E
:1024800084030020001800428C03002094030020E5
:10249000001C004228010020FEE70000034B10B59D
:1024A0001B68002B00D0984710BDC0469C0300203D
:1024B00070B50F490F4CA14204D100F08FF800F025
:1024C000EDFEFEE70C4D00238D42F6D0CA18E81849
:1024D000A24205D3094B8242EFD00949002204E011
:1024E000006804331060F1E704C38B42FCD3E4E7D7
:1024F00000000020A0000020004F0000A0000020ED
:10250000DC09002010B500F066F8002801D100F0C9
:1025100057F810BD014B18607047C0469C0300205F
:10252000014B18687047C046A0030020F7B5134858
:10253000012284461249134C8E68636805689B0E1D
:102540001340019288686268019F920E3A40674684
:102550003F6893420ED1BD420CD186420AD35B192B
:10256000FA254868AD00861B07486B437043000D91
:10257000C018FEBD3D0013000600E3E7A0030020E5
:1025800010E000E000ED00E05555000070B5041EBD
:1025900010D0FFF7CBFF050000F01CF8FFF7C6FFD7
:1025A000054B401B9842F7D9FA23013C9B00ED18DC
:1025B000002CF3D170BDC046E70300007047000057
:1025C00010B5034A13680133136000F0C3FA10BD5D
:1025D000A003002070470020704700001E2270B545
:1025E00046484749436893431C3A134343600823D2
:1025F0008C6923438B61434C434B9C829C8A1443DC
:102600009C82DC681442FCD00124404A1470157886
:10261000254203D055786DB2002DF8DB012494607B
:10262000547864B2002CFBDB394C5460547864B2AB
:10263000002CFBDB8224E4015480547864B2002C2B
:10264000FBDB02249C840E34DD682542FCD0314C37
:10265000DC621024DD682542FCD09D8C2E4C2C437E
:102660009C841024DD682542FCD002249D8C8026A9
:102670002C439C844024DD683542FCD0DD68254233
:10268000F9D01024DD682542FCD0002494605478F1
:1026900064B2002CFBDB214C5460547864B2002CF3
:1026A000FBDB1C6A1E4D2C4080251C621C6AAC435F
:1026B0001C62032393601B4B536053785BB2002B67
:1026C000FBDB0023FF240B72174A4B728B72CB7219
:1026D000164B1A60164B174A1B6811689A065B0165
:1026E000C90E2340520F12020B431343124A1385A3
:1026F000802342681343436070BDC04600400041E0
:10270000000400400C06000000080040000C0040DF
:1027100001050100B905FF7D040A00000007030060
:10272000FFFCFFFF03060100006CDC020400002038
:10273000246080002060800000400042FA21314B7C
:1027400010B51868890001F0FFFF2F4B013898423F
:1027500056D82E492E4A4860C020136A00061B0234
:102760001B0A03431362002407238C600B60802143
:10277000136A09061B021B0A0B431362FC22254B3A
:10278000196A0A431A62FC22196A92010A431A6200
:10279000A022196AD2020A431A62E0B2002101346F
:1027A00000F0EEF8162CF8D11B4B1C005A7852B2F0
:1027B000002AFBDB194A5A80194B1A00597EC909B5
:1027C0000129FBD0E421C90099803F21D970537EB3
:1027D000DB09012BFBD0C02300205B01136190704B
:1027E00000F02EF863785BB2002BFBDB0D4B0E4A3A
:1027F0006380D379DB09012BFBD04123537010BDDB
:10280000FEE7C04604000020FFFFFF0010E000E0EC
:1028100000ED00E000040040000C00401E400000FD
:10282000004000422140000000480042914202D096
:1028300002D98A1AD0407047521A9040FBE7000034
:10284000164A00B51300517EC9090129FBD0013891
:10285000042816D81969124A0A400F211A615A78B9
:102860008A4301F067FF0308060B030011000122F1
:102870000A435A7000BD11000322F9E71100022239
:10288000F6E7F02311691B050B430F211361537801
:102890008B43190002230B435370EBE700400042C7
:1028A000FFFFFFF010B504000E2801D80F34E4B28A
:1028B0000121200000F0DCF81823102163432B4C89
:1028C000E4186156002901D014290DD1284B1800B5
:1028D000DA79D209012AFBD002241A78A2431A70AD
:1028E000C379DB09012BFBD022480300427ED209C9
:1028F000012AFBD01F2402692140A2430A4302613E
:102900005A7ED209012AFBD0022219780A431A7092
:102910005A7ED209012AFBD00222197B0A431A737C
:102920001A7ED207FCD501221A765A7ED209012AD4
:10293000FBD00222197B0A431A731A7ED207FCD5F8
:10294000588B80B25A7ED209012AFBD002211A7814
:102950008A431A705A7ED209012AFBD0064B1A68A4
:10296000064B1968FFF762FF10BDC046B04A000071
:1029700000480042004000420C00002008000020F7
:10298000182330B51D00040045430820204A55197E
:102990002856013014D0032912D808006343D156B9
:1029A000D31801F0C7FE02280E1B5868CB01022184
:1029B000184A9B181A1840321170012282405A603E
:1029C00030BD5868CB010621124A9B181A184032B4
:1029D0001170012282405A609A61F1E75868CB0178
:1029E00006210C4A9B181A184032117001228240AD
:1029F0005A605A61E4E75868CB010221054A9B18E6
:102A00001A1840321170012282409A60D8E7C046FD
:102A1000B04A0000004400411823F0B50824584390
:102A2000114A13181C5701341BD0012635005F686A
:102A30008356BD400D4ADB019A18906805420BD1C0
:102A40000C00601E8441D2194032107834400336A5
:102A5000A400B04320431070044A9B18002901D100
:102A60005D61F0BD9D61FCE7B04A0000004400419B
:102A700018224243F8B52C4E0300B218127A52B213
:102A8000140001320ED0481C00240C280AD801F092
:102A900051FE0720202020202020200B0B0B0B00B4
:102AA000012464422000F8BD092905D10021D8B2D3
:102AB000FFF766FF0024F5E70A2902D1D8B20839EA
:102AC000F6E700240B29EDD1D8B20A39FFF758FFF9
:102AD000E8E718204343F2185568F3562C00134AD0
:102AE000DB016E0817389B18C9B204409E19002CF0
:102AF0000DD00F2430363278090122401143C9B27B
:102B00005B19317040331A7810431870D2E73200E5
:102B10000F27303216785B19BE43314311704033B2
:102B20001A7810431870BDE7B04A00000044004115
:102B300010B50400FFF742FD014B1C6010BDC046FC
:102B4000100000200122024B52421A607047C0461A
:102B500010000020164A10B51368591C26D0013BFE
:102B60001360002B22D172B6124B134A04339342E6
:102B700013D9124A01211000147D0C42FCD02021EF
:102B8000148BFF319B085B0021431183D3610C4BF5
:102B900013800123027D1A42FCD0BFF34F8F094BF3
:102BA000094ADA60BFF34F8FC046FDE710BDC0464B
:102BB000100000200020000003020000004000413F
:102BC00002A5FFFF00ED00E00400FA0500230371F9
:102BD000016070479446F0B59E1E721E9641624693
:102BE000056892072F6836063A4332432A60072564
:102BF00005AC24780068A4012940214342680024E0
:102C0000022B00D05C03114321434160F0BD30B57D
:102C1000C0250368AD031C6812052A402243C02466
:102C20000904A40221401143196003685A6814433F
:102C30005C6030BD0123026811680B4313600368B8
:102C40001A68D207FCD4DA69D207F9D47047022394
:102C5000026811680B4313600268D3699B07FCD4B8
:102C600070470268137E9B0702D40379002BF9D1C9
:102C7000002303717047002203685A83704703687A
:102C8000187E4007C00F70470368187EC009704760
:102C9000802302685B42117E0B4313767047036802
:102CA000588B8007C00F704702230268518B0B437B
:102CB000538370470368187EC007C00F70470368CE
:102CC000188DC0B2704703681A7ED207FCD589B24E
:102CD00019850123037118007047012203689A7552
:102CE0007047012203681A75704700000368214A83
:102CF00030B593422FD0204A93422FD01F4A93429F
:102D00002FD01F4A93422FD01E4A93422FD01E4AE3
:102D100093421FD10E2319220121032599401B48FC
:102D2000C024016099082B40AB40FC359D408900D0
:102D30000918A4000859A843C0259D402B0003434F
:102D40000B518023DB011A43114B5A805A7852B23F
:102D5000002AFBDB30BD09231422DDE70A231522FC
:102D6000DAE70B231622D7E70C231722D4E70D232B
:102D70001822D1E700080042000C00420010004277
:102D80000014004200180042001C004200E100E074
:102D9000000C0040F8B504000F0016001D00FFF7FE
:102DA000A5FF2000FFF746FF1C21BB000B40710769
:102DB0002268090C0B431360842322689375012F4A
:102DC0001AD11021012E00D008390C4B6943186824
:102DD000C00001F0B9FC0722216802408B89520330
:102DE000DB04DB0C13438B81226803049089DB0C2A
:102DF000400B400318439081F8BDC04604000020FA
:102E00000120704710B50368014A1B6A984710BD3E
:102E100013040000FC30006A704787239B00C01831
:102E2000C36880204000C01A70470300FC331A6A50
:102E3000002A03D0DB69C018007D704701204042A2
:102E4000FBE710B504000069FFF7F4FE2200002341
:102E5000FC329361D361136287229200A4186360ED
:102E6000A360E36010BD872310B59B00C218D36830
:102E7000002BFCD10069FFF7F4FE10BD0368002BA6
:102E800002D162B6BFF36F8F7047F0200140303936
:102E9000484248417047F0231B0119408023062017
:102EA0009B0099420AD00133FF330130994205D08B
:102EB000802302385B00994200D0002070470F2029
:102EC00001400020012903D00239481E8141481CDD
:102ED000704700008B23F0B5182685B002919B0047
:102EE0000400C05C330008214343324D1700EB1847
:102EF0005956FFF7BDFD304B0821E05C33004343DA
:102F0000EB185956FFF7B4FD2C4BE25C0393022AF1
:102F100009D11133E05CFF2805D008214643AE19E2
:102F20007156FFF7A5FD8C26B600A05DFF2819D0CD
:102F30000121FFF725FD1822A35D21495A43AB5615
:102F4000AD18DB0158188D21890060501D49012200
:102F50005B188E218900635069688A408F2189003F
:102F600062501A600122029B11002069FFF712FFD4
:102F700039002000FFF78FFF390005002000FFF720
:102F80009EFF390006002000FFF77FFF330000900E
:102F9000290020690122FFF71DFE0B4B2069E25C2E
:102FA000039BE15CFFF733FE2069FFF750FE05B09D
:102FB000F0BDC046B04A00002D0200002F02000004
:102FC00018440041144400412E020000802210B534
:102FD00004005200002101F084FC23000022FC3395
:102FE0005A6020009A60DA6010BD0000F7B51D003D
:102FF00008AB1B780400009309AB1B781600019303
:1030000000234360FA239B008360114B0F000833B9
:1030100003601430FFF7DAFF20002130FF30FFF7A4
:10302000D5FF8B236A469B002761E654094B127833
:10303000E554094B2000E2546A46084B1279E254E9
:103040008C22313BFF3B9200A3541032A354FEBDAF
:10305000104E00002D0200002E0200002F02000082
:10306000F7B5EFF3108300930123019372B6802626
:103070000200FF25019BFC327600013B5C1C0FD057
:10308000D4685F1EB44209D05468015554680134B5
:103090002C405460D4680134D460EEE73B00EDE787
:1030A00068460193FFF7EAFEF7BD13B5EFF310830F
:1030B00000930123019372B6019B5A1E0192002BCB
:1030C00015D00300FC33DA68002A0DD09A68845CBE
:1030D0009A680132D2B29A60DA68013ADA606846D8
:1030E000FFF7CCFE200016BD01246442F7E701245F
:1030F0006846FFF7C3FE6442F4E710B504000069B8
:10310000FFF7CDFD002805D02069FFF7D8FD206925
:10311000FFF7CAFD2069FFF7B2FD00281BD0206928
:10312000FFF7CDFD010020001430FFF799FF8C233D
:103130009B00E35CFF2B0ED02300FC331A6A802334
:103140005B009B1A092B06DC8D238F229B009200CB
:10315000E358A2581A602069FFF7ACFD00280ED092
:1031600087239B00E318DB68002B14D0200021305C
:10317000FF30FFF79AFFC1B22069FFF7A4FD206975
:10318000FFF782FD002805D02069FFF781FD206947
:10319000FFF771FD10BD2069FFF7A3FDEFE7000009
:1031A000F8B5040000690D00FFF784FD87239B003C
:1031B000E618002802D0F368002B34D001278022C3
:1031C000F3685200934223D1EFF310833B4210D1B6
:1031D000174B5B68DB05DB0DF1D0103B5BB2002BBE
:1031E00010DAF13A1340083B9B08124A9B009B18E7
:1031F0001B682069FFF75EFD0028E0D02000FFF784
:103200007CFFDCE79B08C0330B4A9B009B58F0E730
:1032100020002130FF302900FFF722FF2069FFF74F
:103220005CFD0120F8BD29002069FFF74CFDF8E79F
:1032300000ED00E01CED00E000E100E010B504004E
:103240001430FFF732FF8C239B00E35CFF2B0ED082
:103250002300FC331A6A80235B009B1A0A2B06DDCD
:103260008E238F229B009200E358A2581A6010BD53
:10327000F7B506000D000C008B180193019B671B2E
:103280009C4207D0336821781B683000984701348E
:103290000028F3D13800FEBD7047000010B5FFF7DD
:1032A0004DFA01F0DDFAFFF7F7FF0120FFF76EF9A5
:1032B000084C200000F014FF200000F057F9FEF742
:1032C0001DFFFEF723FF044B002BFAD000E000BFE8
:1032D000F7E7C046CC03002000000000704710B59F
:1032E000040001F033F8200010BD0000F0B5822981
:1032F00019D1C3B2294D5A01AA189169284C8001ED
:103300000C40C021890521439161264908334018AA
:103310007021506128685B011A5C8A4311003022D9
:103320000A431A54F0BD0029FCD1C026C1B21B4C7F
:103330004B01E3189A681A4DB6052A4032439A6049
:10334000194A800182185A600A0007272468083247
:103350005201115DB9430F000121394311559F6995
:1033600010493D4040182E439E6158617020115D08
:103370008143080010210143115599680B48A21898
:10338000084080214903014399609968890B8903AA
:103390009960402311790B431371C3E7840800201F
:1033A000FFFFFF8FF8030020B8050020FF3F00F06B
:1033B000EFF3108303600123436072B6704773B567
:1033C000836D0400002B1BD10600A83635786846B3
:1033D000FFF7EEFF019BEDB2013B02D33578EDB272
:1033E000FAE768460193FFF749FD002D01D100205F
:1033F00076BD2300A4331868A0342368C01AF7E709
:103400006846FFF7D5FF22000025019BF432013BFF
:1034100002D31578EDB2FAE768460193FFF72EFD67
:10342000002DE4D02300F0331868EC34E5E7000009
:1034300010B5436D4468DBB25A01A218916809487F
:1034400008330840802149030143916091685B0182
:10345000890B890391602268D318402219790A43A5
:103460001A7110BDFF3F00F0F7B5436D4268DBB243
:10347000190004000831106849014118C979C907C9
:1034800011D55B01D21893689B049B0C0CD12000D2
:10349000FFF7CEFF63681A68636DDBB208335B0128
:1034A000D3187F22DA71F7BDE16D002923D1210005
:1034B000A4310B6023000125AC33E56568465360F9
:1034C000FFF776FF260020002100019BA836013B74
:1034D000F430F5315A1C33D0357002785F1ED2B209
:1034E0000A700A78002A04D120000193FFF7A0FF98
:1034F000E8E73B00EEE72100F0310B600023E365D5
:103500002300603353606846FFF752FF0125260011
:1035100020002100019BF436013BA830F5315A1CF4
:103520000ED0357002785F1ED2B20A700A78002A77
:1035300004D120000193FFF77BFFE8E73B00EEE7B3
:1035400068460193FFF79AFCA4E737B56B46DC1D8C
:1035500000230D00237000F0E3FE210000F06EFE5A
:103560002B681818286020783EBD000000780028DD
:1035700010D00121084B1B681A898A431A8108223E
:10358000198B0A431A830422198B0A431A830022D7
:10359000024B1A607047C046840800207C08002057
:1035A00010B50F4A93699B0B9B039361136802222A
:1035B000FF331A729879823A02439A711A7A920703
:1035C000FCD57F24074A2140937A0800A3431900C1
:1035D000802301439172917A5B420B43937210BD39
:1035E000840800200050004110B50C0000F098FE47
:1035F000210000F056FE002804D1034A93699B0B7A
:103600009B03936110BDC04684080020F8B50D00EF
:10361000832A19D1CBB23B4C5A01A21891693A487E
:10362000AD010840C02189050143916137492068F7
:103630006D187021083355615B011A5C8A431100D3
:1036400040220A431A54F8BD022A55D1304A8B0051
:103650009858002802D003685B699847F82000F06A
:1036600071FE0400274E2B4B466003604022002170
:10367000083001F036F922000023A032A36465650A
:10368000E3642365A365E3655360D3641372136039
:1036900013654C3213725372FF222B0013405901F1
:1036A00071188868184F08330740C02080053843D8
:1036B0008860306807265B01195CAD00B1430E00DD
:1036C0000321314319542300616D606811404901A1
:1036D000411860334B60616D63680A401B6852019A
:1036E0009B180122FF33997A20000A439A72FFF750
:1036F0009FFE074B5C51A6E711002800FFF7F6FD7F
:10370000A1E7C04684080020FFFFFF8FF8030020D8
:10371000D00300204C4E000070B505000124064B7C
:10372000A200D258002A06D0210028000134FFF759
:103730006DFF0A2CF3D170BDA40300200B4BCAB25D
:103740000B488901C9185301C31859619969083296
:10375000890B89039961036852019A180223D37176
:103760005179823B0B4353717047C046F8030020E8
:1037700084080020084B8A00D05810B5002803D0D8
:1037800003689B68984710BDC9B2044B490159189A
:1037900088688004800CF6E7D003002084080020AD
:1037A00010B50C00FFF7E6FF00280CD0064BE4B282
:1037B0001B68083464011C19802362795B4213433F
:1037C00063710223E37110BD84080020F0B51C0072
:1037D0002A4B85B01B6807000D000292002B4AD0CF
:1037E000274B8A00D058002808D0036822005B6865
:1037F000029998470400200005B0F0BD3800FFF79B
:10380000B9FF844204D929003800FFF7B3FF040050
:103810000121EBB21B4E03935B010193F2189368F5
:103820009B0B9B039360019A336802989B18FF33AC
:103830005A7A0A435A72144BA901C918220001F09E
:1038400047F8002CD7D029003800FFF793FF002855
:10385000D1D14021039B326808335B01D31818791A
:10386000014319710121D971019BD318FF339A7A51
:103870000A439A72BFE701246442BCE77C08002037
:10388000D003002084080020B805002013B56B4643
:10389000DC1D22000123FFF799FF012801D12078C8
:1038A00016BD01204042FBE770B5CBB2124A134867
:1038B0005C0189018918021951609168104D083323
:1038C0000D40802149032943402591609168890B6F
:1038D0008903916001685A018A1816793543157178
:1038E00095796D06FCD55B01C918CB79DB07FCD552
:1038F00000198068C0B270BDB8050020840800209F
:10390000FF3F00F070B50D0000211400FFF7CCFF61
:10391000A04200D9200000230349A34203D0CA5C7F
:10392000EA540133F9E770BDB8050020F0B51E0078
:103930003A4B85B01B680F000192002B35D08023D5
:10394000DB019E4231D80025354B8A01D318029302
:10395000002E2CD0334B1B680393FF233B401C00ED
:1039600000930834039B64011C19A379DB0921D05F
:103970002D4B2E49186800F0E7FE2D4B17215843B8
:1039800000F0E2FE2B4BE279920713D4DA5D002AB5
:1039900001D10138F7D20122DA55009B5A01214B9F
:1039A0009B189A69920B92039A6101256D42280037
:1039B00005B0F0BD00221F4B3400DA553F2E09D967
:1039C000009B40245A01174B9B18802299691206CC
:1039D0000A439A6122000199029800F079FF009B46
:1039E000A1045A010F4B890C9B18029A2D195A6198
:1039F0009A69361B920B92030A439A61009B039AC1
:103A000008335B01D3180222DA715979823A0A43EA
:103A10005A71019B1B1901939AE7C0467C0800204C
:103A2000F8030020840800200400002040420F001A
:103A300070110100ED03002070B50D001C000D4B4E
:103A4000AE01F61811003000220000F041FFEDB287
:103A500009496D014D196E61AB69084A2000134098
:103A6000AB61AB69A2049B0B920C9B031343AB614C
:103A700070BDC046F803002084080020FF3F00F01E
:103A8000F7B5104B01901B780F001500002B0CD1DF
:103A90000D4B16001C78002C09D00C4E0C483488B5
:103AA0002018641900F014FF34802800FEBD002E99
:103AB000FBD03A19330000210198FFF7BDFF24180D
:103AC000361AF4E778070020790800207A080020E9
:103AD00079070020F8B50F0016000024012A26D926
:103AE000100000F0E1FE0500380000F0BDFF0323E8
:103AF00002220130400028706B7096420DD939784F
:103B000000290AD0531CDBB20137A9549E4203D0CE
:103B10000232EC54D2B2F0E7320029000548FFF738
:103B2000AFFF441EA041C4B2280000F0C7FE200031
:103B3000F8BDC046CC030020F0B50024012685B0B6
:103B4000184B0F0069461E7005000094FFF7FDFC3E
:103B5000154B01A90B806A3BFF3BCB715A330B72AB
:103B6000009B8C7109334B800E4B4E7108711C7099
:103B70003A00092F0FD00D4F09223E700C4E28003D
:103B800000943480FFF77CFF69462800FFF7DDFCD6
:103B9000328808493C702800FFF772FF012005B009
:103BA000F0BDC04678070020090200007908002017
:103BB0007A0800207907002070B5CE7892B0050011
:103BC0000C00022E0BD18B79C9792C4809021943BC
:103BD000FFF7B2FF411E8841C0B212B070BD00F0C5
:103BE0009FFB210000F03EFB002803D0C117081AFC
:103BF000C00FF2E7012E0ED1E279A37912021A4327
:103C00001F49112A13D8D2B2002A10D02800FFF77A
:103C100037FF0120E1E7032EDFD1A378002B08D185
:103C2000E279A37912021A431649032AEBD90A78DA
:103C3000ECE7022B08D1E279A379120212491A4368
:103C40002800FFF747FFC8E7012B05D1E279A379E8
:103C500012021A430D49F3E7032BBED141220100A2
:103C600001A800F03EFE00F05BFB01A900F00AFB9A
:103C7000E279A37912021A4301A9E1E7CC030020FB
:103C8000884E0000784E0000684E00007C4E000018
:103C9000CBB204495B01C9188B699B0B9B038B61F9
:103CA0007047C0468408002037B5050048780C00EE
:103CB0000B2810D800F03EFD061B0F2B0F4045616E
:103CC000494C5A5D097801AA002906D102231180C6
:103CD0002800FFF7B1FE01203EBD00231380284BD2
:103CE0001B78012B00D1137002230021F0E78A78A2
:103CF0000023012A03D101AA1380224BF0E7204AB6
:103D00001370214A93699B0B9B039361E3E78C78C3
:103D1000012C06D100211B4B01AA1C70117023003D
:103D2000D6E70120002CD7D1154B174A187093699C
:103D30009B0B9B039361CFE789782800FFF730FC4A
:103D4000C9E72800FFF738FFC6E701230F4ACCE791
:103D50000B780020DB06BFD12800FFF7DDFCA2783E
:103D60000A4B0B481A6000F0C3FCCAE70123094A5A
:103D7000BBE78A78074B1A60C3E70020ACE7C04670
:103D8000EC030020F4030020840800207C080020BD
:103D900098090020800800203A4BF7B51E780500EE
:103DA000002E5FD1384C23689A8B12070DD508225C
:103DB00031009A833000FFF799FA10222368FF330D
:103DC000997A0A439A72314B1E6023689A8B520784
:103DD00001D504229A83FF331A7A920603D5202252
:103DE000597A0A435A721A7AD20623D569460800CC
:103DF000274AC0CAC0C0A268920B9203A2604022A8
:103E0000587902435A7160230A7828001A422AD14D
:103E1000FFF74AFF2368FF33002827D080229979D3
:103E200052420A439A711A7A520603D54022597AAD
:103E30000A435A727F2601252368FF331E722F0022
:103E4000236808377F01DB19DB79002B07D0114B82
:103E5000AA00D05800280DD003681B689847013588
:103E6000082DECD1F7BDFFF7BFFBD3E720210A4AAD
:103E70009171D8E72900094800F010FC2368DF1988
:103E8000FE71ECE779080020840800207C080020FF
:103E9000B8050020D0030020FF5000419809002001
:103EA00010B50248FFF778FF10BDC046CC030020D4
:103EB00080235B0003800023436007330372704755
:103EC00083000148C0187047A4030020836C402B76
:103ED00009D03F22036CC154036C013313400364C7
:103EE000836C013383647047F7B505006846FFF7BC
:103EF0005FFA00264022019B013B02D32E6D961BE8
:103F0000FAE768460193FEF7B9FFAB6D6846002BF0
:103F10004FD1FFF74DFA2900019BA831013B5A1CF4
:103F20000CD00C785A1EE4B2002C05D168460193DF
:103F3000FEF7A4FF2000FEBD1300F0E768460193E2
:103F40000024FEF79BFF2A002900A0321368A43149
:103F5000B4420ED0086898420BD92800591CEB18BF
:103F60001160603319780830C9B2FFF7AFFF013430
:103F7000E9E709689942DDD1002313600133AB659D
:103F80006846FFF715FA2F002A000021019BA83789
:103F9000013BF532581CC9D0397010785E1E0028DC
:103FA00005D0117028000193FFF742FAEBE73300C8
:103FB000F0E7FFF7FDF92900019BF431013B5A1CA2
:103FC00006D00C785A1EE4B2002CAFD01300F6E7EE
:103FD000684601930024FEF751FF2A002900EC32C5
:103FE0001368F031B44202D0086898421DD80968BD
:103FF00099429FD1002368461360AB65FFF7D8F95B
:104000002F002A000021019BF437013BF532581C98
:1040100000D18BE7397010785E1E002811D0117026
:1040200028000193FFF704FAEAE72800591CEB186F
:104030001160AC3319780830C9B2FFF747FF01347B
:10404000CBE73300E3E710B50400FFF74DFF206D29
:1040500010BD10B50400FFF747FF236D002B03D000
:10406000E36CE418207A10BD01204042FBE7F7B56D
:1040700017000E000400FFF737FF6846FFF798F9B6
:104080003F2200259446019B013B5A1C19D0BD429A
:1040900015D2226D002A12D00121226D4942002A38
:1040A0000AD06046E26CA218117AE26C013202403A
:1040B000E264226D013A226571550135E7E7013B63
:1040C000E3E768460193FEF7D9FE2800FEBD000035
:1040D000014B024A1A6070478408002000500041DA
:1040E0002023F7B5474A0500D1690F200B43D36160
:1040F000012245490B7813430B70444B19788143D7
:10410000197006211C782143197041490C7822430B
:104110000A701A7802401A70602219780A431A70DD
:104120003C4B3D4A5A805F78FF09FCD13B48FEF783
:10413000F1F901233A4C3B4E2268300011780B43D1
:10414000137080223900520000F0CBFB2268937874
:10415000DB07FCD456621F26334B1B68590B980CA7
:104160009B01314030405B0FB14200D105211F2837
:1041700000D10238072B00D1043B31408901178D53
:1041800001912A4930400F40019939431185118D21
:104190000700B143080038431085118D1803244BE4
:1041A0007F260B4003430C2013850823D1788143DD
:1041B0000B430321D3702268D3788B4301390B431F
:1041C000D370226813783340137004232268167862
:1041D000334313702268C1241389A4008343154814
:1041E000138103591B021B0A0351802303601378B8
:1041F00011481943012311702B70002100F0E8F8D9
:10420000F7BDC04600040040584400413C44004112
:1042100059440041000C004006400000A13E00004F
:104220008408002088080020246080003FF8FFFFF9
:10423000FF8FFFFF00E100E09809002070B50E003D
:1042400000254468002C0BD0236831005B682000F7
:104250009847002802DB2D18E468F3E701256D423A
:10426000280070BD70B50D004468002C08D023688C
:1042700029009B6820009847002802D1E468F4E7F1
:10428000200070BD70B50D004468002C07D0236875
:1042900029002000DB689847E4682D18F5E72C70AA
:1042A00070BD70B50D004468002C08D0236829004B
:1042B0001B6820009847002802D1E468F4E720003A
:1042C00070BDF8B542788B790D00017A9B18040017
:1042D00000208B4222DC6368834219D1656000268E
:1042E00023786A71EA792B719B182370AB79B342FA
:1042F00013D9AB68B7006078DF19FFF7E1FD3B68C1
:10430000013603606378F6B201336370EEE70B00A9
:10431000D9680029FBD1DD60E1E70120F8BD00008C
:1043200070B50126054D064C2B68334203D12000A1
:10433000FFF7BEFD2E60200070BDC046880900203A
:104340008C09002010B500F0AFFA10BD10B500F0D8
:10435000B5FA10BD0020704770B50F26CB1D01398E
:1043600002003240D5B22C0000093034092A00DDA9
:1043700007341C70013B8B42F2D170BD10B50C00AC
:104380000B4B1868FFF7E8FF21000A4B083118684B
:10439000FFF7E2FF2100084B10311868FFF7DCFF40
:1043A0002100064B18311868FFF7D6FF202010BDFA
:1043B0000CA0800040A0800044A0800048A08000A5
:1043C00008B4024B9C46103808BC60477D4300008F
:1043D000704770473F20704713B56B460268D9712C
:1043E0000733546819000122A04716BD70B50A268C
:1043F0000B7892B06E44023305000B703C22002112
:10440000300000F06EFA394801AC0690384824219B
:104410000790062020776846364AA1742281364AE2
:10442000364BA281FD3AFF3A8018C177684623399E
:104430000630C17768460730C17702A8C1770720E8
:10444000F277032608316944C87703A9CE77102193
:104450002B366E443170092621851F3169440E7058
:104460000CA9053E0E7033212380022369440B7092
:1044700006360DA90E7022493536A1863B216E44C1
:10448000307010A86274E27702703D3269446A4469
:104490000B70137040210022E37023716371A373CA
:1044A00041336B44218719705A702B7DC039A3703A
:1044B000A37263770133DBB2A3776A7D0B200D0013
:1044C00068441543C5773120684403703A23501C73
:1044D0006B441870412302320A436B441A70210066
:1044E00042220848FFF7CCFA12B070BD1001042434
:1044F000020605240904000001020000080B000068
:1045000007050000CC03002008B4024B9C4610387D
:1045100008BC6047ED43000070B5027D0B790C00CC
:1045200000259A420BD10B784E78A12B09D1212E70
:1045300005D107221B491C48FFF7A2FA01352800C4
:1045400070BD212BFBD1202E22D107221549164800
:10455000FFF7D8F99622134BD200196891421DD16A
:10456000DB79DB071AD4FA20FEF7E2FA00210E48C5
:10457000FFF78EFB0125232EE1D1E378A2781B0201
:1045800013430A4A002108481360FFF781FBD6E76E
:10459000222EEFD18A78034BDA71DBE7FEF7D2FAED
:1045A000E4E7C04618000020CC03002014000020DF
:1045B00008B4024B9C46103808BC604719450000FF
:1045C00010B508220021024800F08BF910BDC0464A
:1045D0001800002010B5417D006A0131FFF7CAF8CC
:1045E000034B1B6801335A1E9341181810BDC04677
:1045F0002000002010B5417D006A0231FFF7D0F89D
:1046000010BD10B5417D006A0231FFF797F810BD6B
:1046100070B50D00417D0400130002312A00006ACC
:10462000FFF784F9002801D10123636070BD000009
:1046300010B5054C23685A1C04D103685B69984780
:1046400003002060180010BD20000020074A03006E
:10465000106810B5411C03D001235B42136010BDEC
:10466000597D186A0131FFF711F9F8E720000020A1
:1046700010B5FDF755FFF423FF330024984207D906
:10468000044B0A20DC79631E9C41E4B2FDF77EFFF7
:10469000200010BD18000020002070477047000067
:1046A000FA239B0010B583600F4B0022C3820300E6
:1046B000283383610D4B04004260C26118005033FF
:1046C00023610830631D21622060DA778323A362AF
:1046D000813BE36280332363FFF722FE2100103128
:1046E000FFF7EFFD200010BD030200009C4E00000C
:1046F000022110B5094B1A68437D5B01D318FF33C3
:104700009C7A21439972437D0133DBB25B01D3185C
:104710000122FF33997A0A439A7210BD840800205F
:1047200010B502490248FFF7BBFF10BDCC030020C3
:104730009809002002B4714649084900095C490003
:104740008E4402BC7047C046002243088B4274D39B
:1047500003098B425FD3030A8B4244D3030B8B4282
:1047600028D3030C8B420DD3FF22090212BA030C8B
:104770008B4202D31212090265D0030B8B4219D36C
:1047800000E0090AC30B8B4201D3CB03C01A52418C
:10479000830B8B4201D38B03C01A5241430B8B42D4
:1047A00001D34B03C01A5241030B8B4201D30B03BD
:1047B000C01A5241C30A8B4201D3CB02C01A5241E4
:1047C000830A8B4201D38B02C01A5241430A8B42A7
:1047D00001D34B02C01A5241030A8B4201D30B0290
:1047E000C01A5241CDD2C3098B4201D3CB01C01AAA
:1047F000524183098B4201D38B01C01A52414309B4
:104800008B4201D34B01C01A524103098B4201D3A1
:104810000B01C01A5241C3088B4201D3CB00C01A0E
:10482000524183088B4201D38B00C01A5241430886
:104830008B4201D34B00C01A5241411A00D20146AB
:10484000524110467047FFE701B5002000F006F81E
:1048500002BDC0460029F7D076E770477047C046D2
:1048600070B500260C4D0D4C641BA410A64209D156
:10487000002600F011F90A4D0A4C641BA410A64250
:1048800005D170BDB300EB5898470136EEE7B30091
:10489000EB5898470136F2E7880000208800002096
:1048A000880000209C00002010B5034B0100186810
:1048B00000F06AF810BDC0462400002010B5034B7C
:1048C0000100186800F016F810BDC0462400002052
:1048D000002310B59A4200D110BDCC5CC454013302
:1048E000F8E703001218934200D1704719700133A2
:1048F000F9E7000070B50500002910D00C1F2368EF
:10490000002B00DAE418280000F0B5F81D4A1368FF
:10491000002B05D163601460280000F0ADF870BD75
:10492000A34209D9216860188342F3D118685B68F3
:1049300041182160EEE713005A68002A01D0A24214
:10494000F9D919685818A0420BD1206809185818CD
:1049500019608242E0D110685268411819605A60AB
:10496000DAE7A04202D90C232B60D5E72168601852
:10497000824203D1106852684118216062605C6015
:10498000CAE7C046CC090020032370B5CD1C9D4367
:10499000083506000C2D1ED20C25A9421DD830006A
:1049A00000F069F8254A14682100002919D1244C27
:1049B0002368002B03D1300000F044F82060290068
:1049C000300000F03FF8431C2BD10C233000336043
:1049D00000F052F803E0002DDFDA0C2333600020F2
:1049E00070BD0B685B1B19D40B2B03D90B60CC1863
:1049F000256003E04B688C420DD11360300000F05D
:104A00003BF8200007220B30231D9043C31AE7D048
:104A10005A42E250E4E763600C00EFE70C0049689B
:104A2000C3E70323C41C9C43A042E1D0211A3000F9
:104A300000F008F8431CDBD1C7E7C046CC090020D2
:104A4000D0090020002370B5064C05000800236043
:104A500000F014F8431C03D12368002B00D02B6016
:104A600070BDC046D80900200023C25C0133002A73
:104A7000FBD1581E7047704770470000044A136806
:104A8000002B00D1034B1818106018007047C04667
:104A9000D4090020DC090020F8B5C046F8BC08BCE9
:104AA0009E467047F8B5C046F8BC08BC9E467047A5
:104AB0000000000016000000080000001C000000BC
:104AC000FF000004000406000000000017000000C2
:104AD000080000001C000000FF00010401040700A2
:104AE000000000000A000000080000001C00000098
:104AF000120000010001FF00000000000B00000098
:104B0000080000001C000000130001010101FF006B
:104B1000010000000A000000080000001C00000066
:104B2000FF00000500050A00010000000B00000066
:104B3000080000001C000000FF00010501050B003B
:104B40000000000014000000080000002C0000001D
:104B5000FF00020002000400000000001500000039
:104B6000080000002C000000FF0003000300050007
:104B70000000000010000000020000001C00000007
:104B8000FF00000200020000000000001100000011
:104B90000200000004000000FF00FFFFFFFF010013
:104BA0000000000013000000020000001C000000D4
:104BB000FF0001030103FF000000000008000000E7
:104BC000030000001C0000001000000000001000A6
:104BD00000000000090000000300000004000000C5
:104BE0001100FFFFFFFFFF000100000017000000A1
:104BF0000300000004000000FF00FFFFFFFFFF00B4
:104C00000100000016000000030000000400000086
:104C1000FF00FFFFFFFFFF00000000000200000098
:104C200001000000060000000000FFFFFFFFFF0082
:104C3000010000000200000001000000040000006C
:104C40000A00FFFFFFFF0200010000000300000058
:104C500001000000040000000B00FFFFFFFF030045
:104C60000000000004000000010000001C00000023
:104C7000040000000000FF0000000000050000002C
:104C8000010000001C000000050001000100FF0001
:104C90000000000006000000010000000400000009
:104CA0000600FFFFFFFFFF000000000007000000FC
:104CB00001000000040000000700FFFFFFFFFF00ED
:104CC00000000000180000000600000000000000C6
:104CD000FF00FFFFFFFFFF000000000019000000C1
:104CE0000600000000000000FF00FFFFFFFFFF00C4
:104CF0000000000012000000080000000400000096
:104D0000FF00FFFFFFFFFF000000000003000000A6
:104D10000800000004000000FF00FFFFFFFFFF008D
:104D2000000000000C000000030000000000000074
:104D3000FF00FFFFFFFFFF00000000000D0000006C
:104D40000300000000000000FF00FFFFFFFFFF0066
:104D5000000000000E00000008000000000000003D
:104D6000FF00FFFFFFFFFF00000000000F0000003A
:104D70000300000000000000FF00FFFFFFFFFF0036
:104D8000000000001B000000080000000000000000
:104D9000FF00FFFFFFFFFF00000000001C000000FD
:104DA0000800000000000000FF00FFFFFFFFFF0001
:104DB00001000000080000000800000000000000E2
:104DC000FF00FFFFFFFFFF000100000009000000DF
:104DD0000800000000000000FF00FFFFFFFF0900C7
:104DE00000000000000000000800000000000000BB
:104DF000FF00FFFFFFFFFF000000000001000000B8
:104E00000800000000000000FF00FFFFFFFFFF00A0
:104E10000000000000000000A1310000713200001D
:104E20001B2E0000672E0000152E00003D320000F2
:104E30002B2E0000052E0000D52E0000432E000072
:104E4000012E000000000000000000006934000096
:104E50006F4000004740000053400000DD3200007A
:104E6000DF320000BF33000041726475696E6F204D
:104E70004D4B5231303030000403090441726475E7
:104E8000696E6F204C4C430012010002EF0201409A
:104E900041234E80000101020301000000000000D8
:104EA00000000000D943000011460000D543000077
:104EB000F5450000D54500004D4600003146000094
:104EC000D1430000D3430000C145000071460000FB
:104ED00003460000ED430000554300001945000063
:104EE0007D430000F0FFFFFF00000000B14500001F
:104EF0000945000099460000C14300000000000081
:104F00000F00000040420F000A0000000A000000ED
:104F1000FFFFFFFFFFFFFFFF00C2010000000800CE
:104F2000FFFFFFFF2800002000000000000000003D
:104F30000000000000000000000000000000000071
:104F40000000000000000000000000000000000061
:104F50000000000000000000000000000000000051
:104F60000000000000000000000000000000000041
:104F70000000000000000000000000000000000031
:104F80000000000000000000DD20000029210000DA
:104F900019240000D140000021470000B520000086
:04000003000024B124
:00000001FF
